** EXPERIMENTAL (HLL) ** Open Watcom Linker Version 1.6beta1 Limited Availability
Portions Copyright (c) 1985-2002 Sybase, Inc. All Rights Reserved.
Created on:       12/01/07 19:00:18
Warning! W1121: file U:/tmp\ldconv_readline_obj_dda34f080299189350.obj(U:\DEV\python-2.7.2\Modules\readline.c): '_initreadline' has already been exported
Executable Image: build/lib.os2knix-2.7/readline.pyd
creating an OS/2 EMX dynamic link library


                        +------------+
                        |   Groups   |
                        +------------+

Group                           Address              Size
=====                           =======              ====

CGROUP                          0001:00000000        00034bf0
DGROUP                          0002:00000000        00005740



                        +--------------+
                        |   Segments   |
                        +--------------+

Segment                Class          Group          Address         Size
=======                =====          =====          =======         ====

TEXT32                 CODE           CGROUP         0001:00000000   00034bf0
________TEXT           CODE           CGROUP         0001:00034bf0   00000000
DATA32                 DATA           DGROUP         0002:00000000   00003e90
SET1__os2dll           DATA           DGROUP         0002:00003e90   00000004
SET2__os2dll           DATA           DGROUP         0002:00003e94   00000000
SET3__os2dll           DATA           DGROUP         0002:00003e94   00000004
SET1___CTOR_LIST__     DATA           DGROUP         0002:00003e98   00000004
SET2___CTOR_LIST__     DATA           DGROUP         0002:00003e9c   00000000
SET3___CTOR_LIST__     DATA           DGROUP         0002:00003e9c   00000004
SET1___DTOR_LIST__     DATA           DGROUP         0002:00003ea0   00000004
SET2___DTOR_LIST__     DATA           DGROUP         0002:00003ea4   00000000
SET3___DTOR_LIST__     DATA           DGROUP         0002:00003ea4   00000004
SET1___crtinit1__      DATA           DGROUP         0002:00003ea8   00000004
SET2___crtinit1__      DATA           DGROUP         0002:00003eac   00000000
SET3___crtinit1__      DATA           DGROUP         0002:00003eac   00000004
SET1___crtexit1__      DATA           DGROUP         0002:00003eb0   00000004
SET2___crtexit1__      DATA           DGROUP         0002:00003eb4   00000000
SET3___crtexit1__      DATA           DGROUP         0002:00003eb4   00000004
SET1___eh_frame__      DATA           DGROUP         0002:00003eb8   00000004
SET2___eh_frame__      DATA           DGROUP         0002:00003ebc   00000008
SET3___eh_frame__      DATA           DGROUP         0002:00003ec4   00000004
SET1___eh_init__       DATA           DGROUP         0002:00003ec8   00000004
SET2___eh_init__       DATA           DGROUP         0002:00003ecc   00000004
SET3___eh_init__       DATA           DGROUP         0002:00003ed0   00000004
SET1___eh_term__       DATA           DGROUP         0002:00003ed4   00000004
SET2___eh_term__       DATA           DGROUP         0002:00003ed8   00000004
SET3___eh_term__       DATA           DGROUP         0002:00003edc   00000004
SET1___fork_parent1__  DATA           DGROUP         0002:00003ee0   00000004
SET2___fork_parent1__  DATA           DGROUP         0002:00003ee4   00000000
SET3___fork_parent1__  DATA           DGROUP         0002:00003ee4   00000004
SET1___fork_child1__   DATA           DGROUP         0002:00003ee8   00000004
SET2___fork_child1__   DATA           DGROUP         0002:00003eec   00000000
SET3___fork_child1__   DATA           DGROUP         0002:00003eec   00000004
________DATA           DATA           DGROUP         0002:00003ef0   00000000
BSS32                  BSS            DGROUP         0002:00003ef0   00001530
c_common               BSS            DGROUP         0002:00005420   00000320
________BSS            BSS            DGROUP         0002:00005740   00000000


                        +----------------+
                        |   Memory Map   |
                        +----------------+

* = unreferenced symbol
+ = symbol only referenced locally

Address        Symbol
=======        ======

Module: U:\usr\lib\dll0hi.obj({standard input})
0001:00000000* __text
0002:00000000* __data
0002:00000000* ___data_start
0002:00003ef0* ___bss_start
0002:00003e90+ __os2dll
0002:00003e98  ___CTOR_LIST__
0002:00003ea0  ___DTOR_LIST__
0002:00003ea8* ___crtinit1__
0002:00003eb0* ___crtexit1__
0002:00003eb8  ___eh_frame__
0002:00003ec8  ___eh_init__
0002:00003ed4  ___eh_term__
0002:00003ee0+ ___fork_parent1__
0002:00003ee8+ ___fork_child1__
Module: U:/tmp\ldconv_readline_obj_dda34f080299189350.obj(U:\DEV\python-2.7.2\Modules\readline.c)
0001:00000b6e  _initreadline
Module: U:\usr\local446\lib\libc_dll.lib(dllinit.obj)
0001:00001350  _DLL_InitTerm
Module: U:\usr\lib\libend.lib(src/libend/386/endlink386.asm)
0002:00005740  _end
0002:00003ef0  _edata
Module: U:\usr\lib\libend.lib(src/libend/386/end.asm)
0001:00034bf0* _etext
0001:00034bf0* __etext
0000:00000000  WEAK$ZERO
0002:00005740  __end
0002:00003ef0  __edata
Module: U:\extras\lib\libreadline.lib(history.obj)
0002:00005420  _history_offset
0002:00005430  _history_length
0002:00005440+ _history_max_entries
0002:00005450+ _max_input_history
0001:000013b0* _history_set_history_state
0001:000013ec  _using_history
0001:000013fc  _where_history
0001:00001408  _history_set_pos
0001:00001434  _history_list
0001:00001440  _current_history
0001:00001464  _previous_history
0001:00001484  _next_history
0001:000014ac  _history_get
0001:000014d8  _remove_history
0001:00001528* _unstifle_history
0001:00001554* _history_is_stifled
0001:00001560  _history_get_history_state
0001:000015b0* _history_total_bytes
0001:0000163c  _replace_history_entry
0001:000016e8  _free_history_entry
0001:00001734  _clear_history
0001:00001794* _stifle_history
0001:0000184c  _add_history_time
0001:000018a8  _add_history
0001:00001a40* _history_get_time
0002:00000db0  _history_base
Module: U:\extras\lib\libreadline.lib(complete.obj)
0002:00005460  __rl_completion_case_fold
0002:00005470+ _rl_completion_found_quote
0002:00005480+ _rl_completion_quote_character
0002:00005490+ _rl_completion_mark_symlink_dirs
0002:000054a0  __rl_print_completions_horizontally
0002:000054b0  _rl_inhibit_completion
0001:00001a70* _rl_completion_mode
0001:00001b0c* __rl_free_match_list
0001:00002114* __rl_find_completion_word
0001:0000283c* _rl_filename_completion_function
0001:00002db8* _rl_username_completion_function
0001:00002ee8  _rl_completion_matches
0001:0000305c  _rl_menu_complete
0001:00003880* _rl_display_match_list
0001:00003ce8  _rl_complete_internal
0001:0000414c  _rl_insert_completions
0001:00004160  _rl_possible_completions
0001:00004174  _rl_complete
0002:00000ddc* _rl_filename_quoting_desired
0002:00000dd8* _rl_ignore_completion_duplicates
0002:00000dd4  _rl_basic_quote_characters
0002:00000de0* _rl_filename_quoting_function
0002:00000de4  _rl_completion_append_character
0002:00000dc0  __rl_complete_mark_directories
0002:00000dc4  __rl_match_hidden_files
0002:00000dcc  __rl_page_completions
0002:00000dc8  _rl_completion_query_items
0002:00000dd0  _rl_basic_word_break_characters
0002:00003f94  __rl_complete_show_all
0002:00003f98  __rl_complete_show_unmodified
0002:00003fc8* _rl_completer_quote_characters
0002:00003fd4* _rl_filename_completion_desired
0002:00003fdc* _rl_filename_dequoting_function
0002:00003fd8* _rl_ignore_some_completions_function
0002:00003fc4* _rl_completion_word_break_hook
0002:00003fe0* _rl_char_is_quoted_p
0002:00003fd0* _rl_special_prefixes
0002:00003fc0  _rl_completer_word_break_characters
0002:00003fcc* _rl_filename_quote_characters
0002:00003fe4  _rl_completion_suppress_append
0002:00003fe8* _rl_completion_suppress_quote
0002:00003fac  _rl_complete_with_tilde_expansion
0002:00003fa8* _rl_directory_rewrite_hook
0002:00003fa4* _rl_directory_completion_hook
0002:00003fb4  _rl_attempted_completion_function
0002:00003fb8  _rl_attempted_completion_over
0002:00003fbc  _rl_completion_type
0002:00003f9c  __rl_complete_mark_symlink_dirs
0002:00003fb0* _rl_completion_entry_function
0002:00003fa0  _rl_visible_stats
0002:00003f90  _rl_completion_display_matches_hook
Module: U:\extras\lib\libreadline.lib(readline.obj)
0002:000054c0  _rl_mark
0002:000054d0  _rl_end
0002:000054e0  _rl_point
0002:000054f0  _rl_done
0002:00005500+ __rl_in_stream
0002:00005510  __rl_out_stream
0002:00005520+ _rl_executing_keymap
0002:00005530  _rl_dispatching
0002:00005540+ __rl_dispatching_keymap
0002:00005550+ _rl_num_chars_to_read
0002:00005560  _readline_top_level
0002:000055a0  __rl_comment_begin
0001:00004210  __rl_init_line_state
0001:00004240  __rl_set_the_line
0001:00004250* _rl_save_state
0001:00004320* _rl_restore_state
0001:000043f4* __rl_keyseq_cxt_alloc
0001:00004594  _rl_initialize
0001:000047a0* __rl_keyseq_cxt_dispose
0001:000047ac* __rl_keyseq_chain_dispose
0001:000047d8* __rl_dispatch_subseq
0001:00004be4  __rl_dispatch
0001:00004d0c  __rl_dispatch_callback
0001:00004dec  __rl_internal_char_cleanup
0001:00004eac  _readline_internal_char
0001:00004ffc  _readline_internal_teardown
0001:00005104  _readline_internal_setup
0001:000051f0  _rl_set_prompt
0001:0000526c* _readline
0002:00000dfc  __rl_keymap
0002:00000e04  _rl_insert_mode
0002:00000e00  _rl_editing_mode
0002:00000e1c  __rl_bind_stty_chars
0002:00000e18  __rl_convert_meta_chars_to_ascii
0002:00000e0c  _rl_arg_sign
0002:00000e08  _rl_numeric_arg
0002:00000e10  __rl_eof_char
0002:00000df0* _rl_library_version
0002:00000df4* _rl_readline_version
0002:00000df8* _rl_gnu_readline_p
0002:00000e14  __rl_bell_preference
0002:00004168  _rl_line_buffer
0002:0000416c  _rl_line_buffer_len
0002:0000413c  _rl_prompt
0002:00004128  _rl_readline_state
0002:0000412c  _rl_last_func
0002:00004148  _rl_key_sequence_length
0002:00004130  _rl_instream
0002:00004134  _rl_outstream
0002:00004154  _rl_pending_input
0002:00004170  __rl_kscxt
0002:00004174  __rl_parsing_conditionalized_out
0002:00004158  _rl_terminal_name
0002:0000415c  __rl_horizontal_scroll_mode
0002:00004164  _rl_erase_empty_line
0002:00004120  __rl_last_command_was_kill
0002:0000414c  _rl_startup_hook
0002:00004138  _readline_echoing_p
0002:00004144* _rl_already_prompted
0002:00004150  _rl_pre_input_hook
0002:00004140  _rl_visible_prompt_length
0002:0000417c  __rl_meta_flag
0002:00004124  _rl_explicit_arg
0002:00004160  __rl_mark_modified_lines
0002:00004178  __rl_output_meta_chars
Module: U:\extras\lib\libreadline.lib(histfile.obj)
0001:00005620  _write_history
0001:00005644* _append_history
0001:00005668  _history_truncate_file
0001:000058c0* _read_history_range
0001:00005b3c  _read_history
0002:000041c0* _history_write_timestamps
Module: U:\extras\lib\libreadline.lib(bind.obj)
0002:000055b0+ _rl_binding_keymap
0001:00005b60  _rl_bind_key
0001:00005bc4  _rl_bind_key_in_map
0001:00005bf8* _rl_unbind_key
0001:00005c14* _rl_unbind_key_in_map
0001:00005c38* _rl_unbind_function_in_map
0001:00005c78* _rl_untranslate_keyseq
0001:00005e54* _rl_function_of_keyseq
0001:00005f44* _rl_get_keymap_name
0001:00005f78* _rl_set_keymap
0001:00005f8c* _rl_get_keymap
0001:00005f98  _rl_set_keymap_from_edit_mode
0001:00005fd4* _rl_get_keymap_name_from_edit_mode
0001:00006828* _rl_macro_dumper
0001:00006850  _rl_dump_macros
0001:00006a2c* _rl_get_keymap_by_name
0001:00006cf0* _rl_variable_dumper
0001:00006e10  _rl_dump_variables
0001:00006e5c* _rl_variable_value
0001:00006f1c* _rl_list_funmap_names
0001:00006f70* _rl_invoking_keyseqs_in_map
0001:0000724c* _rl_invoking_keyseqs
0001:00007294* _rl_variable_bind
0001:00007628* _rl_named_function
0001:000076dc* _rl_function_dumper
0001:000078a8  _rl_dump_functions
0001:000078f4* _rl_unbind_command_in_map
0001:00007958* _rl_translate_keyseq
0001:00007f54* _rl_generic_bind
0001:00008104* _rl_macro_bind
0001:0000817c* _rl_set_key
0001:000081a8* _rl_bind_keyseq_in_map
0001:000081d4* _rl_bind_keyseq_if_unbound_in_map
0001:00008244  _rl_bind_keyseq_if_unbound
0001:00008268* _rl_bind_key_if_unbound
0001:00008298* _rl_bind_key_if_unbound_in_map
0001:000082c4* _rl_bind_keyseq
0001:00008338  _rl_parse_and_bind
0001:00008ca8  _rl_read_init_file
0001:00008cf4  _rl_re_read_init_file
0001:00008d30* _rl_add_defun
0002:00000e3c  _rl_readline_name
0002:00000e20* __rl_possible_control_prefixes
0002:00000e30* __rl_possible_meta_prefixes
Module: U:\extras\lib\libreadline.lib(display.obj)
0001:00009210  _rl_on_new_line
0001:0000926c  _rl_forced_update_display
0001:000092a0  _rl_character_len
0001:00009308  _rl_reset_line_state
0001:00009334  _rl_save_prompt
0001:000093c8  __rl_current_display_line
0001:0000940c  __rl_clear_screen
0001:00009440  __rl_clear_to_eol
0001:000094a8  __rl_erase_entire_line
0001:00009520  __rl_move_vert
0001:000095d8  __rl_clean_up_for_exit
0001:0000981c  __rl_strip_prompt
0001:00009850  __rl_make_prompt_for_search
0001:00009938  __rl_erase_at_end_of_line
0001:000099b0  __rl_move_cursor_relative
0001:00009a7c  __rl_update_final
0001:00009b54  _rl_restore_prompt
0001:00009c0c  __rl_redisplay_after_sigwinch
0001:00009d6c  _rl_clear_message
0001:00009da0  _rl_expand_prompt
0001:00009efc  _rl_message
0001:00009f98* _rl_show_char
0001:0000a224  _rl_on_new_line_with_prompt
0001:0000ab14  _rl_redisplay
0002:00000e50  _rl_redisplay_function
0002:00004294* __rl_last_v_pos
0002:00004290  __rl_last_c_pos
0002:00004298  __rl_vis_botlin
0002:0000428c  _rl_display_prompt
0002:00004280  _rl_display_fixed
0002:00004284* __rl_suppress_redisplay
0002:00004288  __rl_want_redisplay
Module: U:\extras\lib\libreadline.lib(text.obj)
0001:0000ba30  __rl_fix_point
0001:0000ba84  _rl_beg_of_line
0001:0000ba98  _rl_end_of_line
0001:0000baac  _rl_do_lowercase_version
0001:0000bab4  __rl_set_mark_at_pos
0001:0000bad4  _rl_set_mark
0001:0000bb04  _rl_exchange_point_and_mark
0001:0000bb4c  __rl_char_search_internal
0001:0000bc10  _rl_backward_byte
0001:0000bc68  _rl_forward_byte
0001:0000bce4  _rl_forward_char
0001:0000bcf0* _rl_forward
0001:0000bcfc  _rl_backward_char
0001:0000bd08* _rl_backward
0001:0000bd6c  _rl_backward_char_search
0001:0000bdfc  _rl_char_search
0001:0000be54  _rl_backward_word
0001:0000bee0  _rl_forward_word
0001:0000c114  _rl_capitalize_word
0001:0000c128  _rl_downcase_word
0001:0000c13c  _rl_upcase_word
0001:0000c150  _rl_newline
0001:0000c1ec  _rl_arrow_keys
0001:0000c2ac  _rl_refresh_line
0001:0000c2f4  _rl_clear_screen
0001:0000c334  _rl_replace_line
0001:0000c39c  _rl_delete_text
0001:0000c474  _rl_delete_horizontal_space
0001:0000c514  _rl_delete
0001:0000c5a0  __rl_rubout_char
0001:0000c684  _rl_delete_or_show_completions
0001:0000c6b8  _rl_rubout_or_delete
0001:0000c6ec  _rl_insert_text
0001:0000c834  _rl_transpose_chars
0001:0000c8cc  _rl_transpose_words
0001:0000ca04  _rl_insert_comment
0001:0000caa8  __rl_insert_char
0001:0000cb9c* __rl_overwrite_rubout
0001:0000cc90  _rl_rubout
0001:0000cce4  _rl_tab_insert
0001:0000cd40  _rl_quoted_insert
0001:0000cdb8  __rl_overwrite_char
0001:0000ce1c  _rl_insert
0001:0000ce48  __rl_replace_text
Module: U:\extras\lib\libreadline.lib(keymaps.obj)
0001:0000ce90* _rl_discard_keymap
0001:0000cee0  _rl_make_bare_keymap
0001:0000cf10* _rl_make_keymap
0001:0000cf5c* _rl_copy_keymap
0002:00000e60  _emacs_standard_keymap
0002:00001e80  _emacs_ctlx_keymap
0002:00001670  _emacs_meta_keymap
0002:00002690  _vi_movement_keymap
0002:00002ea0  _vi_insertion_keymap
Module: U:\extras\lib\libreadline.lib(signals.obj)
0001:0000cf90  _rl_free_line_state
0001:0000cfbc  _rl_clear_signals
0001:0000d0f0  _rl_cleanup_after_signal
0001:0000d1e8  _rl_set_signals
0001:0000d374* _rl_reset_after_signal
0002:000036b0  _rl_catch_signals
0002:000036b4  _rl_catch_sigwinch
Module: U:\extras\lib\libreadline.lib(callback.obj)
0002:000055c0+ _rl_linefunc
0001:0000d4d0* __rl_callback_data_dispose
0001:0000d4e8  __rl_callback_data_alloc
0001:0000d510  _rl_callback_handler_remove
0001:0000d5d8  _rl_callback_read_char
0001:0000d8c8  _rl_callback_handler_install
0002:00004580  __rl_callback_func
0002:00004584  __rl_callback_data
Module: U:\extras\lib\libreadline.lib(rltty.obj)
0001:0000d900* _rl_tty_unset_default_bindings
0001:0000d9a0  __rl_restore_tty_signals
0001:0000da1c  __rl_disable_tty_signals
0001:0000dafc* _rltty_set_default_bindings
0001:0000db70  _rl_tty_set_default_bindings
0001:0000db7c* _rl_stop_output
0001:0000dba4  _rl_restart_output
0001:0000dc70* _rl_deprep_terminal
0001:0000dcf4  _rl_prep_terminal
0002:000036c0  _rl_prep_term_function
0002:000036c4  _rl_deprep_term_function
Module: U:\usr\local446\lib\gcc\i386-pc-os2-emx\4.4.6\libgcc.lib(emx-ctordtor.obj)
0001:0000e030  ___ctordtorTerm
0001:0000e062  ___ctordtorInit
Module: U:\extras\lib\libreadline.lib(xmalloc.obj)
0001:0000e0a0* _xfree
0001:0000e10c  _xrealloc
0001:0000e158  _xmalloc
Module: U:\extras\lib\libreadline.lib(histexpand.obj)
0002:000055d0+ _history_inhibit_expansion_function
0001:0000e654* _history_tokenize
0001:0000e710  _history_arg_extract
0001:0000e8d0* _get_history_event
0001:0000ec90* _history_expand
0002:00003728* _history_word_delimiters
0002:00003720* _history_expansion_char
0002:00003721* _history_subst_char
0002:00003724* _history_no_expand_chars
0002:000046f0  _history_comment_char
0002:000046f4* _history_quotes_inhibit_expansion
Module: U:\extras\lib\libreadline.lib(util.obj)
0001:00010310* __rl_digit_p
0001:00010324* __rl_digit_value
0001:00010330* __rl_lowercase_p
0001:0001035c* __rl_pure_alphabetic
0001:00010388* __rl_to_lower
0001:000103b8* __rl_to_upper
0001:000103e8* __rl_uppercase_p
0001:00010414* __rl_savestring
0001:00010448  __rl_qsort_string_compare
0001:00010464  __rl_strindex
0001:000104dc  _rl_copy_text
0001:0001052c  _rl_tilde_expand
0001:00010644  _rl_extend_line_buffer
0001:00010694  _rl_tty_status
0001:000106a4  __rl_abort_internal
0001:00010700  _rl_abort
0001:0001070c  _rl_alphabetic
0002:00004770* __rl_allow_pathname_alphabetic_chars
Module: U:\extras\lib\libreadline.lib(tilde.obj)
0001:0001081c* _tilde_expand_word
0001:00010a14  _tilde_expand
0002:00003730* _tilde_additional_prefixes
0002:00003734* _tilde_additional_suffixes
0002:00004780* _tilde_expansion_preexpansion_hook
0002:00004784* _tilde_expansion_failure_hook
Module: U:\extras\lib\libreadline.lib(terminal.obj)
0002:000055e0  __rl_screenheight
0002:000055f0  __rl_screenwidth
0002:00005600+ __rl_term_backspace
0002:00005610+ _rl_prefer_env_winsize
0002:00005620  __rl_screenchars
0002:00005630  __rl_term_clreol
0002:00005640  __rl_term_cr
0002:00005650  __rl_term_clrpag
0002:00005660  __rl_term_IC
0002:00005670  __rl_term_ic
0002:00005680  __rl_term_ei
0002:00005690  __rl_term_im
0002:000056a0  __rl_term_DC
0002:000056b0  __rl_term_dc
0002:000056c0  __rl_term_up
0002:000056d0+ __rl_term_pc
0002:000056e0  __rl_enable_keypad
0002:000056f0+ __rl_term_goto
0002:00005700+ __rl_term_ip
0001:00010d60* _rl_get_screen_size
0001:00010d84* __rl_set_cursor
0001:00010f68  __rl_output_character_function
0001:00010dec  __rl_control_keypad
0001:00010e28  __rl_enable_meta_key
0001:00010e5c  _rl_ding
0001:00010ed4  _rl_crlf
0001:00010ef4  __rl_backspace
0001:00010f84  __rl_output_some_chars
0001:00010fb0* _rl_get_termcap
0001:000110d4* __rl_get_screen_size
0001:00011298  __rl_init_terminal_io
0001:00011730* _rl_reset_terminal
0001:0001175c* __rl_set_screen_size
0001:000117d4* _rl_set_screen_size
0001:000117e0  _rl_resize_terminal
0001:0001182c* _rl_reset_screen_size
0002:00003750  __rl_term_autowrap
0002:00003754  __rl_enable_meta
0002:00004790  __rl_terminal_can_insert
Module: U:\extras\lib\libreadline.lib(input.obj)
0001:00011990  __rl_any_typein
0001:000119a8  __rl_unget_char
0001:00011a0c  __rl_pushed_input_available
0001:00011a24* _rl_set_keyboard_input_timeout
0001:00011a3c  _rl_stuff_char
0001:00011aac  _rl_execute_next
0001:00011ac8  _rl_clear_pending_input
0001:00011ae4* _rl_getc
0001:00011c84  __rl_input_available
0001:00011d30  __rl_input_queued
0001:00011f8c  _rl_read_key
0001:0001206c  __rl_insert_typein
0002:00003760* _rl_getc_function
0002:000048e0* _rl_event_hook
Module: U:\extras\lib\libreadline.lib(undo.obj)
0001:00012150* __rl_fix_last_undo_of_type
0001:00012188  _rl_free_undo_list
0001:000121dc  _rl_do_undo
0001:00012390  _rl_undo_command
0001:000123bc  _rl_revert_line
0001:00012404  _rl_add_undo
0001:00012440  _rl_end_undo_group
0001:00012474  _rl_begin_undo_group
0001:000124a8  _rl_modifying
0002:00004b28  _rl_undo_list
0002:00004b20  __rl_doing_an_undo
0002:00004b24  __rl_undo_group_level
Module: U:\extras\lib\libreadline.lib(macro.obj)
0001:00012530* __rl_push_executing_macro
0001:00012564  __rl_with_macro_input
0001:00012590* _rl_push_macro_input
0001:0001259c  _rl_call_last_kbd_macro
0001:00012628  _rl_end_kbd_macro
0001:0001267c  _rl_start_kbd_macro
0001:000126fc  __rl_kill_kbd_macro
0001:00012764  __rl_pop_executing_macro
0001:000127d4  __rl_next_macro_key
0001:00012840  __rl_add_macro_char
0002:00004b30  _rl_executing_macro
Module: U:\extras\lib\libreadline.lib(misc.obj)
0002:00005710  __rl_argcxt
0001:000128d0  __rl_reset_argument
0001:00012900  _rl_emacs_editing_mode
0001:00012928  __rl_set_insert_mode
0001:00012938  _rl_overwrite_mode
0001:00012964  _rl_vi_editing_mode
0001:00012998* _rl_replace_from_history
0001:000129f0  _rl_maybe_save_line
0001:00012a6c  _rl_maybe_replace_line
0001:00012ad0  __rl_free_history_entry
0001:00012b10  __rl_free_saved_history_line
0001:00012b38  _rl_maybe_unsave_line
0001:00012b94  _rl_get_next_history
0001:00012cc0  _rl_get_previous_history
0001:00012df4  _rl_beginning_of_history
0001:00012e14  _rl_end_of_history
0001:00012e30  __rl_start_using_history
0001:00012e58* _rl_discard_argument
0001:00012e94  __rl_arg_overflow
0001:00012ef8  __rl_arg_getchar
0001:00012f30* __rl_arg_dispatch
0001:00013194  _rl_universal_argument
0001:000130c0  __rl_arg_callback
0001:00013170* __rl_arg_init
0001:000131bc  _rl_digit_argument
0002:00003770  __rl_history_saved_point
0002:00004b94  __rl_saved_line_for_history
0002:00004b90  __rl_history_preserve_point
Module: U:\extras\lib\libreadline.lib(vi_mode.obj)
0001:00013220  __rl_vi_initialize_line
0001:00013248  __rl_vi_reset_last
0001:00013278  __rl_vi_set_last
0001:00013298* _rl_vi_start_inserting
0001:000132c8  _rl_vi_fWord
0001:00013350  _rl_vi_bWord
0001:000133f8  _rl_vi_eWord
0001:000134d0  _rl_vi_fword
0001:000135fc  _rl_vi_bword
0001:00013820  _rl_vi_eword
0001:000139b0  _rl_vi_append_mode
0001:000139dc  _rl_vi_insertion_mode
0001:000139f8  _rl_vi_check
0001:00013a1c* _rl_vi_bracktype
0001:00013ad0  _rl_vi_goto_mark
0001:00013b60  _rl_vi_set_mark
0001:00013bac  _rl_vi_end_word
0001:00013c04  _rl_vi_next_word
0001:00013c74  _rl_vi_prev_word
0001:00013ce4  _rl_vi_replace
0001:00013e38  _rl_vi_overstrike
0001:00013d88  _rl_vi_overstrike_delete
0001:00014fb0  _rl_vi_movement_mode
0001:00013d6c  _rl_vi_eof_maybe
0001:00013e84  _rl_vi_match
0001:00013fc0  _rl_vi_char_search
0001:0001415c  _rl_vi_back_to_indent
0001:000141b0  _rl_vi_first_print
0001:000141c0  _rl_vi_insert_beg
0001:000141f4  _rl_vi_delete
0001:00014274  _rl_vi_rubout
0001:00014364  _rl_vi_change_char
0001:00014434  _rl_vi_change_case
0001:0001454c  __rl_vi_textmod_command
0001:00014574  _rl_vi_redo
0001:00014624* _rl_vi_domove
0001:00014990  _rl_vi_yank_to
0001:00014a58  _rl_vi_change_to
0001:00014c48  _rl_vi_subst
0001:00014c94  _rl_vi_delete_to
0001:00014d50  _rl_vi_column
0001:00014d84  _rl_vi_append_eol
0001:00014dcc  _rl_vi_put
0001:00014e40  _rl_vi_arg_digit
0001:00014f30  __rl_vi_done_inserting
0001:00015008  _rl_vi_tilde_expand
0001:00015054  _rl_vi_complete
0001:00015138  _rl_vi_search
0001:0001519c  _rl_vi_search_again
0001:000151dc  _rl_vi_fetch_history
0001:0001524c  _rl_vi_yank_arg
0001:0001528c  _rl_vi_undo
0002:00003780  __rl_vi_last_command
Module: U:\extras\lib\libreadline.lib(funmap.obj)
0002:00005720  _funmap
0002:00005730+ _funmap_program_specific_entry_start
0001:000152d0  _rl_add_funmap_entry
0001:00015358  _rl_initialize_funmap
0001:000153b0  _rl_funmap_names
Module: U:\extras\lib\libreadline.lib(nls.obj)
0001:00015fcc  __rl_init_eightbit
Module: U:\extras\lib\libreadline.lib(shell.obj)
0001:000160d0  _sh_unset_nodelay_mode
0001:00016130  _sh_get_home_dir
0001:0001614c  _sh_get_env_value
0001:0001616c  _sh_set_lines_and_columns
0001:00016208  _sh_single_quote
Module: U:\extras\lib\libreadline.lib(isearch.obj)
0001:00016280  __rl_scxt_dispose
0001:000164d8* __rl_isearch_dispatch
0001:00016e4c  _rl_reverse_search_history
0001:00016e40  _rl_forward_search_history
0001:00016b2c  __rl_search_getchar
0001:00016b50  __rl_isearch_callback
0001:00016b94  __rl_scxt_alloc
0002:00004d24  __rl_iscxt
0002:00004d20  __rl_isearch_terminators
Module: U:\extras\lib\libreadline.lib(parens.obj)
0001:00016e70* _rl_set_paren_blink_timeout
0001:00016e88* _rl_insert_close
0001:00017074  __rl_enable_paren_matching
0002:00003790  _rl_blink_matching_paren
Module: U:\extras\lib\libreadline.lib(mbutil.obj)
0001:00017130* __rl_find_next_mbchar
0001:0001713c* __rl_find_prev_mbchar
0002:000037a0  _rl_byte_oriented
Module: U:\extras\lib\ncurses.lib(lib_tputs.obj)
0001:000175b0* __nc_outch
0001:00017150  _tputs
0001:000174b0* _delay_output
0001:00017580  __nc_flush
0001:00017610  _putp
0002:00004d50  _PC
0002:00004d52  _ospeed
0002:00004d54* __nc_nulls_sent
Module: U:\extras\lib\ncurses.lib(lib_tgoto.obj)
0001:00017640  _tgoto
Module: U:\extras\lib\libreadline.lib(kill.obj)
0001:00017660* _rl_set_retained_kills
0001:0001773c  _rl_yank_last_arg
0001:0001781c  _rl_yank_nth_arg
0001:00017840  _rl_yank
0001:00017884  _rl_yank_pop
0001:00017c1c  _rl_copy_backward_word
0001:00017c44  _rl_copy_forward_word
0001:00017c6c  _rl_copy_region_to_kill
0001:00017c80  _rl_kill_text
0001:00017cd0  _rl_unix_line_discard
0001:00017d24  _rl_unix_filename_rubout
0001:00017e1c  _rl_unix_word_rubout
0001:00017efc  _rl_kill_full_line
0001:00017f3c  _rl_backward_kill_word
0001:00017f9c  _rl_kill_word
0001:00018004  _rl_kill_region
0001:00018048  _rl_kill_line
0001:000180b4  _rl_backward_kill_line
Module: U:\extras\lib\libreadline.lib(search.obj)
0001:000183b8  _rl_history_search_backward
0001:00018430  _rl_history_search_forward
0001:00018574  _rl_noninc_reverse_search_again
0001:000185a8  _rl_noninc_forward_search_again
0001:0001879c  __rl_nsearch_callback
0001:0001894c  _rl_noninc_reverse_search
0001:00018984  _rl_noninc_forward_search
0002:00004dc0  __rl_nscxt
Module: U:\tmp\ldconv_libgcc_so_d_a_dda34f080299196640.lib(emx-eh.obj)
0001:000189f5  ___ehInit
0001:000189c0* ___ehTerm
Module: U:\extras\lib\libreadline.lib(histsearch.obj)
0001:00018be0  _history_search_prefix
0001:00018c04  _history_search
0001:00018c28* _history_search_pos
0002:00004e50  _history_search_delimiter_chars
Module: U:\extras\lib\ncurses.lib(lib_termcap.obj)
0001:00018c90  _tgetent
0001:000191a0  _tgetstr
0001:000192a0  _tgetflag
0001:00019320  _tgetnum
0002:00004e60  _UP
0002:00004e64  _BC
Module: U:\extras\lib\ncurses.lib(lib_cur_term.obj)
0001:000193b0  _set_curterm
0001:00019410  _del_curterm
0002:00004ed0  _cur_term
Module: U:\extras\lib\ncurses.lib(lib_data.obj)
0002:00004ee0* _stdscr
0002:00004ee4* _curscr
0002:00004ee8* _newscr
0002:00004eec* __nc_screen_chain
0002:00004ef0  _SP
Module: U:\extras\lib\ncurses.lib(lib_napms.obj)
0001:00019470  _napms
Module: U:\extras\lib\ncurses.lib(lib_baudrate.obj)
0001:00019560  __nc_baudrate
0001:000195b0  __nc_ospeed
0001:000195f0  _baudrate
Module: U:\extras\lib\ncurses.lib(lib_tparm.obj)
0001:00019650* __nc_tparm_analyze
0001:00019980  _tparm
0002:00004f20* __nc_tparm_err
Module: U:\extras\lib\ncurses.lib(lib_setup.obj)
0001:0001acb0  __nc_setupterm
0001:0001b150* _use_env
0001:0001b160* __nc_get_locale
0001:0001b190* __nc_unicode_locale
0001:0001b200* __nc_locale_breaks_acs
0001:0001b360* _setupterm
0002:00003830* _ttytype
0002:00005110  _LINES
0002:00005114  _COLS
0002:00005118* _TABSIZE
Module: U:\extras\lib\ncurses.lib(trim_sgr0.obj)
0001:0001b4d0  __nc_trim_sgr0
Module: U:\extras\lib\ncurses.lib(codes.obj)
0001:0001c030  _boolcodes
0001:0001c170  _numcodes
0001:0001c6f0  _strcodes
Module: U:\extras\lib\ncurses.lib(free_ttype.obj)
0001:0001cd70  __nc_free_termtype
0001:0001ce30* _use_extended_names
0002:00003950  __nc_user_definable
Module: U:\extras\lib\ncurses.lib(doalloc.obj)
0001:0001ce50  __nc_doalloc
Module: U:\extras\lib\ncurses.lib(comp_error.obj)
0001:0001cee0  __nc_warning
0001:0001cff0  __nc_err_abort
0001:0001d100  __nc_syserr_abort
0001:0001d210* __nc_get_source
0001:0001d220* __nc_set_source
0001:0001d230  __nc_set_type
0001:0001d290  __nc_get_type
0002:00005120  __nc_suppress_warnings
0002:00005124  __nc_curr_line
0002:00005128  __nc_curr_col
Module: U:\extras\lib\ncurses.lib(read_entry.obj)
0001:0001d2c0* __nc_read_termtype
0001:0001dd20* __nc_read_file_entry
0001:0001ddd0  __nc_read_entry
Module: U:\extras\lib\ncurses.lib(fallback.obj)
0001:0001e0a0  __nc_fallback
Module: U:\extras\lib\ncurses.lib(lib_ttyflags.obj)
0001:0001e0b0* __nc_get_tty_mode
0001:0001e130  __nc_set_tty_mode
0001:0001e1b0* _def_shell_mode
0001:0001e230  _def_prog_mode
0001:0001e2b0* _reset_prog_mode
0001:0001e360* _reset_shell_mode
0001:0001e430* _savetty
0001:0001e4b0* _resetty
Module: U:\extras\lib\ncurses.lib(name_match.obj)
0001:0001e530  __nc_name_match
0001:0001e620  __nc_first_name
Module: U:\extras\lib\ncurses.lib(getenv_num.obj)
0001:0001e690  __nc_getenv_num
Module: U:\extras\lib\ncurses.lib(comp_parse.obj)
0001:0001e6f0* __nc_delink_entry
0001:0001e7a0* __nc_read_entry_source
0001:0001e990* __nc_resolve_uses2
0001:00020290* __nc_free_entries
0001:000202c0  __nc_free_entry
0001:000202f0* __nc_entry_match
0001:00020490* __nc_resolve_uses
0002:00003960* __nc_check_termtype2
0002:00003964* __nc_check_termtype
0002:00005190  __nc_head
0002:00005194* __nc_tail
Module: U:\usr\local446\lib\gcc\i386-pc-os2-emx\4.4.6\libgcc.lib(_alloca.obj)
0001:000204d0  __alloca
Module: U:\extras\lib\ncurses.lib(access.obj)
0001:00020510* __nc_rootname
0001:000205b0* __nc_is_abs_path
0001:000205f0  __nc_pathlast
0001:00020640* __nc_basename
0001:00020690  __nc_access
0001:00020760  __nc_is_dir_path
0001:000207b0* __nc_is_file_path
Module: U:\extras\lib\ncurses.lib(db_iterator.obj)
0001:00020850  __nc_next_db
0001:00020990* __nc_tic_dir
0001:000209e0* __nc_keep_tic_dir
0001:00020a30  __nc_last_db
0001:00020a70* __nc_first_db
Module: U:\extras\lib\ncurses.lib(setbuf.obj)
0001:00020b80  __nc_set_buffer
Module: U:\extras\lib\ncurses.lib(lib_options.obj)
0001:00020c40* _curs_set
0001:00020d00* _idlok
0001:00020d60* _idcok
0001:00020db0* _halfdelay
0001:00020e00* _nodelay
0001:00020e30* _notimeout
0001:00020e50* _wtimeout
0001:00020e70* _keypad
0001:00020f00* _meta
0001:00020f70* _typeahead
0001:00020f90* _has_key
0001:00021010  __nc_keypad
Module: U:\extras\lib\ncurses.lib(comp_scan.obj)
0001:00021390  __nc_get_token
0001:00022190  __nc_panic_mode
0001:00021cb0* __nc_trans_string
0001:000221b0  __nc_reset_input
0001:00022210  __nc_push_token
0002:000051f0  __nc_syntax
0002:000051f4* __nc_curr_file_pos
0002:000051f8  __nc_comment_start
0002:000051fc  __nc_comment_end
0002:00005200  __nc_start_line
0002:00005204  __nc_curr_token
0002:00005210* __nc_disable_period
Module: U:\extras\lib\ncurses.lib(parse_entry.obj)
0001:00022f00  __nc_parse_entry
0001:00023690* __nc_capcmp
Module: U:\extras\lib\ncurses.lib(alloc_entry.obj)
0001:00024e70  __nc_wrap_entry
0001:000253e0  __nc_merge_entry
0001:000254e0  __nc_init_entry
0001:00025600  __nc_copy_entry
0001:00025670  __nc_save_str
Module: U:\extras\lib\ncurses.lib(alloc_ttype.obj)
0001:00025710  __nc_align_termtype
0001:000259f0  __nc_copy_termtype
Module: U:\extras\lib\ncurses.lib(home_terminfo.obj)
0001:000266d0  __nc_home_terminfo
Module: U:\extras\lib\ncurses.lib(lib_has_cap.obj)
0001:00026760  _has_ic
0001:000267d0  _has_il
Module: U:\extras\lib\ncurses.lib(lib_raw.obj)
0001:00026820* _raw
0001:000268e0  _cbreak
0001:00026990* _qiflush
0001:000269f0* _noraw
0001:00026ab0* _nocbreak
0001:00026b50* _noqiflush
0001:00026bb0* _intrflush
Module: U:\extras\lib\ncurses.lib(init_keytry.obj)
0001:00026c30  __nc_init_keytry
0002:00003990* __nc_tinfo_fkeys
Module: U:\extras\lib\ncurses.lib(unctrl.obj)
0001:00027490  _unctrl
Module: U:\extras\lib\ncurses.lib(lib_trace.obj)
0002:00005310  __nc_tracing
Module: U:\extras\lib\ncurses.lib(comp_captab.obj)
0001:000295b0  __nc_info_hash_table
0001:0002c1f0  __nc_cap_hash_table
0001:0002d210  __nc_capalias_table
0001:0002d450  __nc_infoalias_table
0001:0002d4b0  __nc_get_table
0001:0002d4d0* __nc_get_hash_table
Module: U:\extras\lib\ncurses.lib(comp_hash.obj)
0001:0002d4f0  __nc_find_entry
0001:0002d590  __nc_find_type_entry
Module: U:\extras\lib\ncurses.lib(captoinfo.obj)
0001:0002d6d0  __nc_captoinfo
0001:0002e980* __nc_infotocap
Module: U:\extras\lib\ncurses.lib(strings.obj)
0001:00031350  __nc_str_init
0001:00031380* __nc_str_null
0001:000313b0* __nc_str_copy
0001:000313e0  __nc_safe_strcat
0001:00031450* __nc_safe_strcpy
Module: U:\extras\lib\ncurses.lib(visbuf.obj)
0001:000314e0* __nc_visbuf2
0001:00031580  __nc_visbuf
0001:000315a0* __nc_visbufn
Module: U:\extras\lib\ncurses.lib(names.obj)
0001:00031830* _boolnames
0001:00031bd0  _boolfnames
0001:00031d50* _numnames
0001:00032050  _numfnames
0001:000328d0  _strnames
0001:00034310  _strfnames
Module: U:\extras\lib\ncurses.lib(key_defined.obj)
0001:00034a20  _key_defined
Module: U:\extras\lib\ncurses.lib(add_tries.obj)
0001:00034a60  __nc_add_to_try


                        +----------------------+
                        |   Imported Symbols   |
                        +----------------------+

Symbol                              Module
======                              ======

___libc_ForkRegisterModule          libc064
___init_dll                         libc064
___libc_Back_termDll                libc064
___libc_ForkDeregisterModule        libc064
__atfork_callback                   libc064
__Py_NoneStruct                     python27
_PyArg_ParseTuple                   python27
_PyOS_snprintf                      python27
_PyCallable_Check                   python27
_PyExc_TypeError                    python27
_PyErr_SetString                    python27
_PyString_FromString                python27
_PyGILState_Ensure                  python27
_PyList_New                         python27
_PyList_SetItem                     python27
_PyErr_Clear                        python27
_PyGILState_Release                 python27
_PyObject_CallFunction              python27
_PyInt_AsLong                       python27
_PyErr_Occurred                     python27
_PyExc_ValueError                   python27
_PyErr_Format                       python27
_PyInt_FromLong                     python27
__errno                             libc064
_PyExc_IOError                      python27
_PyErr_SetFromErrno                 python27
_PyErr_NoMemory                     python27
_Py_InitModule4                     python27
_PyOS_ReadlineFunctionPointer       python27
_Py_FatalError                      python27
_PyString_AsString                  python27
_PyOS_InputHook                     python27
__PyOS_ReadlineTState               python27
_PyEval_RestoreThread               python27
_PyErr_CheckSignals                 python27
_PyEval_SaveThread                  python27
_PyMem_Malloc                       python27
__CRT_init                          libc064
__CRT_term                          libc064
___libc_GLocaleCtype                libc064
___stderrp                          libc064
___stdoutp                          libc064
___stdinp                           libc064
__std_free                          libc064
__std_strdup                        libc064
__std_malloc                        libc064
__std_strcpy                        libc064
__std_setlocale                     libc064
__std_getenv                        libc064
__std_fileno                        libc064
__std_select                        libc064
__std_strncpy                       libc064
__std_strcmp                        libc064
___ctordtorTerm1                    libc064
___ctordtorInit1                    libc064
__std_time                          libc064
__std_snprintf                      libc064
__std_atol                          libc064
__std_qsort                         libc064
__std_strncmp                       libc064
__std_strchr                        libc064
__std_strpbrk                       libc064
_getpwnam                           libc064
__std_stat                          libc064
__std_lstat                         libc064
__std_strrchr                       libc064
__std_readdir                       libc064
__std_strnicmp                      libc064
__std_closedir                      libc064
__std_opendir                       libc064
__std_setpwent                      libc064
__std_getpwent                      libc064
__std_endpwent                      libc064
__scrsize                           libc064
__std_access                        libc064
__std_putc                          libc064
__read_kbd                          libc064
__std_fwrite                        libc064
__std_fflush                        libc064
__std_fprintf                       libc064
_getpwuid                           libc064
__std_sigsetjmp                     libc064
__std_fputs                         libc064
__std_open                          libc064
__std_write                         libc064
__std_close                         libc064
__std_fstat                         libc064
__std_read                          libc064
__std_atoi                          libc064
__std_stricmp                       libc064
__std_sprintf                       libc064
__std_strcat                        libc064
__std_fputc                         libc064
__std_vsnprintf                     libc064
__std_sigemptyset                   libc064
__std_sigaction                     libc064
__std_sigprocmask                   libc064
__std_sigdelset                     libc064
__std_signal                        libc064
__std_getpid                        libc064
__std_kill                          libc064
__std_abort                         libc064
__std_tcsetattr                     libc064
__std_tcgetattr                     libc064
__std_tcflow                        libc064
__std_sigaddset                     libc064
___deregister_frame                 gcc446
___register_frame_table             gcc446
__std_exit                          libc064
__std_realloc                       libc064
__std_strcoll                       libc064
__std_siglongjmp                    libc064
__std_isatty                        libc064
__std_ioctl                         libc064
__std_fcntl                         libc064
__std_getuid                        libc064
__std_setenv                        libc064
__std_strlen                        libc064
__std_nanosleep                     libc064
__std_cfgetospeed                   libc064
__std_calloc                        libc064
__std_nl_langinfo                   libc064
__std_strstr                        libc064
__std_vfprintf                      libc064
__std_strncat                       libc064
__std_memcpy                        libc064
__std_memset                        libc064
__std_strtol                        libc064
__std_setvbuf                       libc064
__std_ftell                         libc064
__std_fgets                         libc064
__std_setmode                       libc064
__std_sscanf                        libc064


                        +--------------------+
                        |   Libraries Used   |
                        +--------------------+

U:\extras\lib\libreadline.lib
U:\extras\lib\ncurses.lib
U:\tmp\ldconv_python2_7_dll_a_dda34f080299190c68.lib
U:\usr\local446\lib\gcc\i386-pc-os2-emx\4.4.6\libgcc.lib
U:\tmp\ldconv_libgcc_so_d_a_dda34f080299196640.lib
U:\usr\lib\libc_alias.lib
U:\usr\local446\lib\libc_dll.lib
U:\usr\lib\libend.lib


                        +-----------------------+
                        |   Linker Statistics   |
                        +-----------------------+

Stack size:  0000 (0.)
Memory size:  0003a330 (238384.)
Link time: 00:00.12
